:030000000236D3F2
:0C36D30078FFE4F6D8FD75816C02371A10
:1012E40020000A3C2E2E2E3E004950436F6E6E6540
:1012F40063745245510A004950436F6E6E656374BE
:10130400000A49504E6F41434B210A003E432C567C
:101314002C52432CC0E4E0EFF2E5F020D1E8EDEAF2
:10132400EEEC49500A003E432C4D41432C2530320B
:1013340062583A25303262583A25303262583A259A
:10134400303262583A25303262583A253032625887
:101354002C4D414320E0E4F0E5F10A003E432C56D5
:1013640045522C20332E3220EEF220257320257393
:101374002CC2E5F0F1E8FF20495020ECEEE4F3EB59
:10138400FF0A00417072203235203230303800318B
:10139400363A31363A3433003E432C4C442C5052C6
:1013A4004F473A20202020202020202020202020C9
:1013B4002020202020202020202020202020202029
:1013C4002020202020202020202020202020202019
:1013D4002020202020202020202020202020202009
:1013E40020202020202020202CC4E0F2E020EFF058
:1013F400EEF8E8E2EAE828F4E0E9EB290A003E2AFC
:101404002C312CCEF1EDEEE2EDFBE520EFE0F0E047
:10141400ECE5F2F0FB20F1E5F2E5E2EEE3EE20E8A4
:10142400EDF2E5F0F4E5E9F1E00A003E412C41304B
:10143400312C2562752E2562752E2562752E256246
:10144400752C495020E0E4F0E5F120E0E4E0EFF20F
:10145400E5F0E00A003E412C4130322C2562752E25
:101464002562752E2562752E2562752C495020E063
:10147400E4F0E5F120EEF1ED2E20F1E5F0E2E5F007
:10148400E00A003E412C4130332C2562752E256242
:10149400752E2562752E2562752C495020E0E4F0E6
:1014A400E5F120F0E5E72E20F1E5F0E2E5F0E00AD1
:1014B400003E412C4130342C2562752E2562752E58
:1014C4002562752E2562752CCCE0F1EAE020F1E569
:1014D400F2E80A003E412C4130352C2562752E2558
:1014E40062752E2562752E2562752CD8EBFEE70AEF
:1014F400003E2A2C312CC4EEEF2E20EFE0F0E0EC7D
:10150400E5F2F0FB20F1E5F2E5E2EEE3EE20E8EDB2
:10151400F2E5F0F4E5E9F1E00A003E422C53303103
:101524002C2562752CC6E4E0F2FC20E7E0EFF0EE37
:10153400F1E020F1EEE5E4E8EDE5EDE8FF20EEF280
:1015440020F1E5F0E2E5F0E00A003E422C533032AF
:101554002C2562752CCEE1ECE5ED20F120F1E5F0CF
:10156400E2E5F0EEEC20E1E5E720EAE2E8F2E0ED86
:10157400F6E8E90A003E422C5330332C2562752CE0
:10158400CFE5F0E5E7E0EFF3F1EA20EFF0E820EF54
:10159400EEF2E5F0E520F1E2FFE7E820F120F1E5E5
:1015A400F0E2E5F0EEEC0A003E454E440A000A443F
:1015B400756D7058202020202030302030312030AC
:1015C400322030332030342030352030362030374C
:1015D4002030382030392030412030422030432020
:1015E4003044203045203046000A3A003A20000AB0
:1015F400000A44756D7044202020202030302030B3
:101604003120303220303320303420303520303611
:1016140020303720303820303920304120304220EB
:10162400304320304420304520304600457272203B
:101634006B657900526420656570726F6D0A0052A3
:1016440064204D454D0A00526420436F64650A00CE
:10165400577269746520436F64650A004465627556
:10166400674950204F4E0A0044656275674950200F
:101674004F46460A00446562756755736572204F8C
:101684006E0A00446562756755736572204F46465D
:101694000A0044656275674D7367204F6E0A004403
:1016A400656275674D7367204F46460A00436F6E47
:1016B400666967206C6F636B210A00577220656549
:1016C40070726F6D0A0020536176652065657072D3
:1016D4006F6D210A00457272204D414321004C6F09
:1016E40061643E3E002A003C4130313D003C4130C3
:1016F400323D003C4130333D003C4130343D003C00
:101704004130353D003C21003C5330313D003C53D9
:1017140030323D003C5330333D003C5330353D00C6
:061724003C5330363D008D
:0640B10001690001670037
:10411700C28E438910E4F58B758DB8D2ABD28E224F
:03001B0002364367
:10364300C0E0C083C082C0D0C28E758B00758DB8B8
:10365300201E0675A61E75A6E10567D21AE56960E8
:10366300020569E568D3940140021568056CE56CB1
:10367300540F7048D226E56C543F7012D2189066EE
:103683008BE0600A04F0E0D394B44002D21E90664B
:1036930086E0600204F0906104E0600214F090663A
:1036A3008CE0D394014003E014F0301D02056AE579
:1036B3006BD394644004D21E8002056BE566D394F9
:1036C3000140021566D28ED0D0D082D083D0E032B2
:10085F00C2AFC2237D027C007F071240948F27E531
:10086F0027646060097D017F6012400ED223E4FD92
:10087F00FC7F0B1240948F27E52730E6097D04E4B7
:10088F00FF124032D2237D017C007F071240948FEC
:10089F0027E5277008FD7FFF12400ED22330230378
:1008AF00126000C288C2A8C2AA7589001235A7902B
:1008BF0063497403F0A374CCF0E4906348F01233EF
:1008CF0078123FE8C21E123CDFD223C225C2249009
:1008DF0065767408F09062B47424F0E4A3F090632A
:1008EF003EE09062B6F090633FE09062B7F09063A5
:1008FF0040E09062B8F0906341E09062B9F090638D
:10090F0042E09062BAF0906343E09062BBF075688A
:10091F0001E4906577F0C21FC220C221C2222023BA
:10092F0018AF27FE7D031231BCE4FF1234F77E129D
:10093F007FE4E4FBFDFC122EC990668BE06003742C
:10094F0001F0E4906104F0F56A906575F0F56B12B3
:10095F00411775A70775A61E75A6E1D2AFE4F56B13
:10096F00906104E07003121FE890668CE0B40111EF
:10097F009080007410F0E490668CF0D223C224C2F1
:10098F0025908008E0F52730E405D21F7410F0E5BC
:10099F002730E508D2219080087420F0E52730E653
:1009AF0008D2209080087440F0E56AC39403401980
:1009BF00908002E4F0908001F0908000F0E56A945E
:1009CF00064006E4F56A123CDF9080A0E070031247
:1009DF0039FB9080B8E07003123A759080D0E070C8
:1009EF0003123BC1908000E07013301F10122FD004
:1009FF00906331EFF0D394004003120036908002E1
:100A0F00E07006908000E06005D21D02096CC21DE7
:100A1F00E4F56A906104E0600302096C20231290F0
:100A2F006578E0600C7E127FE61230D4E490657832
:100A3F00F03021121229DE906331EFF0D394004091
:100A4F0005E0FF120032202003020BD012256A901E
:100A5F006331EFF0700302096C906375E054BF24AB
:100A6F007F7003020B39147003020B112402600311
:100A7F00020B722023077E127FED1230D420270342
:100A8F00020BD090634DE0FF7006906351E0606100
:100A9F00906682E0FEB50722A3E0FF90634EE0B5BB
:100AAF000718906684E0FF90634FE0B5070C9066DF
:100ABF0085E0FF906350E06F6037906351E06E60A8
:100ACF0003020BD0906683E0FF906352E06F6003E8
:100ADF00020BD0906684E0FF906353E06F600302D7
:100AEF000BD0906685E0FF906354E06F6003020BBC
:100AFF00D0C21B9065777401F012416F75680102C7
:100B0F000BD090668BE060037401F090667AE0FF83
:100B1F00906377E06F6003020BD090667AE004F089
:100B2F00E4F568906575F0020BD0301B03020BD013
:100B3F00906344E0700302096C906355740AF012DD
:100B4F0040CDD21BE4F568906575F090668604F091
:100B5F00E4906679F0A3F02023677E127FFB1230BA
:100B6F00D4805E90668BE060037401F0301B52906E
:100B7F006375E020E74B906377E0FF906679E0FEC6
:100B8F006F600D906681E07007EE146F7033801305
:100B9F00906679E004F0906331E0FFD39404400352
:100BAF00123E1A9060007482F0A37401F090637784
:100BBF00E0906002F07E607F007D031237E602094D
:100BCF006C201B03020CE8E5687068123F37EF607A
:100BDF00237E647F75906476E02404FD1237E690DF
:100BEF006681E07009906355E0F56802096CE4F5E1
:100BFF006802096C906686E0D3943C40369066811B
:100C0F00E0703090668604F0123442E4906475F020
:100C1F00A37412F090667AE0906477F0A374FDF0FD
:100C2F0090610563A20190647963A2017F12122281
:100C3F00B8809E12415D8F27E527B40115906000A3
:100C4F007483F0E4A3F07E607F007D021237E6022A
:100C5F00096CE527D39401401C9060007483F0A3C6
:100C6F007401F0E52724FEA3F07E607F007D031260
:100C7F0037E602096CE5686401600302096C906550
:100C8F0075E004F02023077E137F051230D49063A4
:100C9F0055E0C394C85004E02432F0906575E0C36A
:100CAF009405400DC21BE4906577F012416F020965
:100CBF006C7C667D82906349E0FAA3E0FB7F0212B1
:100CCF0039777E647F75906476E02404FD1237E6F1
:100CDF00906355E0F56802096CE5686401600302F2
:100CEF00096C906577E014604624FE60421470032F
:100CFF00020DDB2404600302096CE4F56A2027135C
:100D0F009065777404F0906575E05401F075680193
:100D1F0002096C9080027410F0E4906577F0906592
:100D2F007504F07568FA90668274FFF002096C9092
:100D3F006682E07003020DC59064757480F0906454
:100D4F00777401F0E4A3F0A304F0A37430F0A3745C
:100D5F007BF0E4F527747C2527F582E43464F58372
:100D6F00747DF0747D2527F582E43464F583E4F017
:100D7F00E5272407906476F07C667D82906349E0D6
:100D8F00FAA3E0FB7F021239777E647F75E5272493
:100D9F0009FD1237E6906681E0601B1240CDD21B31
:100DAF00E4F568906575F090668604F0E4906679D6
:100DBF00F0A3F002096C302707E4906577F0800606
:100DCF009065777404F07568FA02096C908002746C
:100DDF0010F0756805906575E06401FFF090657718
:100DEF007401F0EF7019906351E06013FCA3E0FD04
:100DFF00A3E0FEA3E0FF906682121EAA02096C9088
:100E0F00634DE0FCA3E0FDA3E0FEA3E0FF9066824C
:080E1F00121EAA02096C80FEFC
:010E270022A8
:10003600906376E0B444047F0180027F009063758C
:10004600E0B447047E0180027E00EE5F604A906362
:100056003EE0906377F090633FE0906378F09063C2
:1000660040E0906379F0906341E090637AF09063AA
:1000760042E090637BF0906343E090637CF0906392
:10008600767452F09062AE63A2019080A863A201DA
:100096007F061222B8020855906331E0C3940850D7
:1000A6000302085E90633EE0FF906377E06F6003B3
:1000B60002085E90633FE0FF906378E06F600302A2
:1000C600085E906340E0FF906379E06F600302088A
:1000D6005E906341E0FF90637AE06F600302085E22
:1000E600906342E0FF90637BE06F600302085E90DE
:1000F6006343E0FF90637CE06F600302085E9063F9
:1001060076E0B444159062AEE0B4FF0E63A20190AF
:1001160080A863A2017F061222B890668BE0600376
:100126007401F090668C7464F09063767452F0906B
:100136006375E0646D60030202637BFF7A137910D6
:1001460012178C7BFF7A13792A90633EE0F530A371
:10015600E0F531A3E0F532A3E0F533A3E0F534A3EF
:10016600E0F53512178C7530FF75311375328775CA
:1001760033FF7534137535937BFF7A137960121745
:100186008C7BFF7A13799C12178C7BFF7A14790289
:1001960012178C7BFF7A14792F906344E0F530A315
:1001A600E0F531A3E0F532A3E0F53312178C7BFFBF
:1001B6007A14795990634DE0F530A3E0F531A3E068
:1001C600F532A3E0F53312178C7BFF7A147987900A
:1001D6006351E0F530A3E0F531A3E0F532A3E0F595
:1001E6003312178C7BFF7A1479B590633AE0F530B9
:1001F600A3E0F531A3E0F532A3E0F53312178C7BCB
:10020600FF7A1479D8906336E0F530A3E0F531A390
:10021600E0F532A3E0F53312178C7BFF7A1479F5FB
:1002260012178C7BFF7A15791EA227E433F530125C
:10023600178C7BFF7A15794E906681E0F5301217A0
:100246008C7BFF7A15797990668BE0F53012178CE6
:10025600122C9D7BFF7A1579AC12178C2290637550
:10026600E0644C70737E157FB2FBFDFC122EC990C4
:10027600637DE0F528A3E0F529E4F52BE5289063F6
:100286007FF0A3E529F07E157FED7C637D7F7B0201
:10029600122EC9E4F52A852982852883E0FF747F1A
:1002A600252AF582E43463F583EFF00529E5297004
:1002B600020528052AE52AB410DC7E157FF07C634A
:1002C6007D7F7B10122EC9052BE52BC3941040AC05
:1002D6007E157FF31230D422906375E0646C7060F3
:1002E600F52C7E157FF5FBFDFC122EC9E4F52BE4FB
:1002F60090637FF0A3E52CF07E157FED7C637D7F18
:100306007B02122EC9E4F52AA82CE6FF747F252A63
:10031600F582E43463F583EFF0052C052AE52AB46B
:1003260010E67E157FF07C637D7F7B10122EC9055B
:100336002BE52BC3940840B77E157FF31230D422E9
:10034600906375E0644B7061F52A7467252AF5821F
:10035600E43463F583E060327467252AF582E43479
:1003660063F583E0F460237467252AF582E4346339
:10037600F583E0FF747D252AF582E43463F583E096
:10038600B50710052AE52AB408C09061047432F056
:100396000208559063757421F03023030208557ED8
:1003A600167F301230D4020855906375E0B4521AA5
:1003B6002023077E167F381230D49063757472F04E
:1003C6007E637F757D0812375F22906375E064490E
:1003D60070452023077E167F431230D490637DE05C
:1003E600F528A3E0F529E4F52A852982852883E006
:1003F600FF747F252AF582E43463F583EFF005293F
:10040600E52970020528052AE52AB480DC7E637F8B
:10041600757D8A12375F22906375E06443704620CB
:1004260023077E167F4B1230D490637DE0F528A318
:10043600E0F529E4F52A852982852883E493FF746B
:100446007F252AF582E43463F583EFF00529E52953
:1004560070020528052AE52AB480DB7E637F757D58
:100466008A12375F22906375E0645A70532023071F
:100476007E167F541230D490637DE0F528A3E0F514
:10048600297C637D7F7B80AF29AE28123F03E4F58C
:100496002A852982852883E493FF747F252AF5829D
:1004A600E43463F583EFF00529E529700205280594
:1004B6002AE52AB480DB7E637F757D8A12375F2248
:1004C600906375E06444600302055790637DE0FF26
:1004D60064447003020855EFB4310CC2237E167FC4
:1004E600601230D402085590637DE0B4300CD223FC
:1004F6007E167F6C1230D402085590637DE0B432CC
:100506000CD2247E167F791230D402085590637D72
:10051600E0B4330CC2247E167F871230D40208550D
:1005260090637DE0B4340CD2257E167F961230D4CB
:1005360002085590637DE0B4350CC2257E167FA374
:100546001230D402085590637DE0FF124103020881
:1005560055906104E070132023077E167FB1123098
:10056600D49063757421F00208559061047432F0DA
:10057600906375E0FFB45104C2AF80FEEF6457701C
:10058600452023077E167FBF1230D490637EE0900D
:100596006331F0E4F52A906331E0FFE52AC39F401A
:1005A60003020855747F252AF582E43463F583E057
:1005B600FF90637DE0252A24ADF582E43461F5835E
:1005C600EFF0052A80D0906375E06453600302065D
:1005D600792023077E167FCA1230D490633EE0FF4F
:1005E6009061B6E06F703C90633FE0FF9061B7E0CA
:1005F6006F7030906340E0FF9061B8E0B5072490DB
:100606006341E0FF9061B9E0B50718906342E0FFEF
:100616009061BAE0B5070C906343E0FF9061BBE0E0
:100626006F60169063757421F03023030208557EBF
:10063600167FD91230D4020855E4F52AE4F56B7416
:10064600AD252AF582E43461F583E0FDAF2A123F39
:1006560095052AE52AC394FE40E2C2AFE4907FF0F6
:10066600F0A3F0907FFD74AAF0A374FFF0A3745575
:10067600F080FE906375E0644F704C90637DE0F50A
:1006860028A3E0F529E5294528700A2023077E16C8
:100696007FE21230D42023077E167FE91230D4E49D
:1006A600F52A747F252AF582E43463F583E08529EB
:1006B60082852883F00529E52970020528052AE5A3
:1006C6002AB480DE020855906375E0FFB445219098
:1006D600637DE0FDA3E0907FF0CDF0A3EDF0C2AF27
:1006E600907FFD74AAF0A374FFF0A37455F080FE0A
:1006F600EF6465600302085E90637DE0FFA3E0900F
:100706007FF0CFF0A3EFF0E4F528F529D3907FF141
:10071600E09529907FF0E095284021E4F56B2529A6
:10072600FFE5283478FE7B80AD29AC28123F0374A0
:10073600802529F529E43528F52880D07E167FEB1B
:1007460012386DEF4E6020120003906344EFF012F2
:100756000003906345EFF0120003906346EFF0123A
:100766000003906347EFF07E167FF112386DEF4E6F
:10077600602012000390634DEFF012000390634E69
:10078600EFF012000390634FEFF0120003906350F6
:10079600EFF07E167FF712386DEF4E6020120003E1
:1007A600906351EFF0120003906352EFF0120003D2
:1007B600906353EFF0120003906354EFF07E167FC0
:1007C600FD12386DEF4E602012000390633AEFF091
:1007D60012000390633BEFF012000390633CEFF0CE
:1007E60012000390633DEFF07E177F0312386DEF22
:1007F6004E6020120003906336EFF0120003906300
:1008060037EFF0120003906338EFF01200039063A5
:1008160039EFF0E4F52AE4F56BE52A04FF74362592
:100826002AF582E43463F583E0FD123F95052AE557
:100836002AC3944340E0C2AFE4907FF0F0A3F09067
:100846007FFD74AAF0A374FFF0A37455F080FE7EBA
:08085600637F757D0812375F16
:01085E002277
:103E9500AE07EEC39430400BEED394395005EE24B3
:103EA500D0FF22EEC39461400BEED394665005EE2D
:103EB50024A9FF22EEC39441400BEED3944650054E
:083EC500EE24C9FF22AF062222
:1040E9009062ADE004F070069062ACE004F090627A
:0A40F900ACE0FEA3E0FF123DD82268
:100003001240E9123E95EFC454F0FEC0061240E9D7
:08001300123E95D0E02FFF2200
:103C8200E4906A82F01240E9906A83EFF0C39430C4
:103C92004018E0FFD394395011906A82E02405F570
:103CA20082E43461F583EFF08011906A82E02405AA
:103CB200F582E43461F583E4F0800C906A82E004DA
:103CC200F0E0D3940840BE752B00752C00752D00D2
:0C3CD200E4F52E7B017A6179051223C60F
:013CDE0022C3
:04386D008E2D8F2EDF
:103871009062ACE4F0A374FFF01240E9EF606EF4E3
:10388100606B852E82852D83E493B507EC752F013E
:10389100E52E252FF582E4352DF583E493602590FF
:1038A10062ADE0252FFF9062ACE03400FE123DD8FE
:1038B100E52E252FF582E4352DF583E493B5070434
:1038C100052F80CCE52E252FF582E4352DF583E4F7
:1038D1009370A6E52F24FFFFE434FFFE9062ADE074
:1038E1002FF09062ACE03EF07E007F0122E4FEFF0B
:0138F10022B4
:103378007E177F0912386DEF4E70037F01227E178A
:103388007F0C12386DEF4E600C1240E9EF24D02408
:10339800FF92278002D2277E177F1212386DEF4ED8
:1033A800600C1240E9EF24D0906681F08005E4902B
:1033B8006681F07E177F1812386DEF4E600C124050
:1033C800E9EF24D090668BF08005E490668BF07E60
:1033D800177F1E12386DEF4E600C1240E9EF24D0B3
:1033E80024FF92198002C21990633E63A20190667D
:1033F8007B63A2017F061222B830193B7E177F2417
:1034080012386DEF4E603012000390667BEFF012B9
:10341800000390667CEFF012000390667DEFF012D7
:10342800000390667EEFF012000390667FEFF012C3
:0A3438000003906680EFF07F002291
:103D9100906576E0C3947C503D906576E0FE04F03A
:103DA10074B42EF582E43462F583EFF0BF0A2790F4
:103DB1006576E0FF04F074B42FF582E43462F58394
:103DC100E4F0906576E0FF1238F29065767408F0C1
:073DD1009062B5E004F0224E
:103CDF009080007480F090633663A201F583F582C3
:103CEF0063A2017F081222B890633E63A201908005
:103CFF008863A2017F0A1222B8908092E4F0A37425
:103D0F0032F0A37401F0906348E0FF9080B1F0901F
:103D1F0080E1EFF09080957455F0A3F090800074DF
:093D2F0001F090800974F0F0220B
:1039FB00908009E04410F09080A0E0706C9080A162
:103A0B007482F09080A874FFF0A3F0A3F0A3F07F72
:103A1B00039080AEEFF07FCBA3EFF07F039080ACF1
:103A2B00EFF0A374CBF09080007402F0906A7212E6
:103A3B001EB600000000906A72E0908040F0906A21
:103A4B0073E0908041F0906A74E0908042F0906A4D
:103A5B0075E0908043F0A3E4F0A3F0A3F0A3F09003
:093A6B008018F0A3F0A3F0A3F011
:013A7400222F
:103BC100908009E04440F09080D17482F090634984
:103BD100E0FF9080DEF090634AE0FF9080DFF0909C
:103BE10080027402F0906A76121EB6000000009006
:103BF1006A76E0908058F0906A77E0908059F09072
:103C01006A78E090805AF0906A79E090805BF0A346
:103C1100E4F0A3F0A3F0A3F0908030F0A3F0A3F0C0
:023C2100A3F00E
:013C2300227E
:103A7500908009E04420F09080B8E0706C9080B9A7
:103A85007482F07F039080C6EFF07FCDA3EFF07FC7
:103A9500039080C4EFF0A374CDF09080C074FFF064
:103AA500A3F0A3F0A3F09080017402F0906A7A125B
:103AB5001EB600000000906A7AE090804CF0906A93
:103AC5007BE090804DF0906A7CE090804EF0906AAB
:103AD5007DE090804FF0A3E4F0A3F0A3F0A3F09075
:093AE5008024F0A3F0A3F0A3F08B
:013AEE0022B5
:103977008C288D29A907EAFDE975F018A424ACFF66
:10398700E5F034808F82F583EDF0EBFDE975F018F3
:10399700A4FFAEF024ACFBEE34808B82F583A3ED5D
:1039A700F08529828C83E0FDEF24A8FFEE3480FEAA
:1039B7008F82F583EDF08529828C83A3E08F828E39
:1039C70083A3F0852982852883A3A3E0FDE975F009
:1039D70018A424A8FFE5F03480FE8F82F583A3A303
:1039E700EDF08529828C83A3A3A3E08F828E83A326
:0439F700A3A3F02274
:06375F008D2DAB07AA0648
:10376500908000E030E5079065787401F022906A5A
:1037750072E0FCA3E0FDA3E0FEA3E0F5318E308D01
:103785002F8C2EAE02AF038E838F8263A201E530AC
:10379500540744C0F58385318263A201AF2D1223FE
:1037A5002AE4FCFDFEE531252DF531EE3530F53009
:1037B500ED352FF52FEC352EF52E908040E52EF0CA
:1037C500A3E52FF0A3E530F0A3E531F09080007478
:1037D50020F0AF31AE30AD2FAC2E906A72121EAA1A
:0137E50022C1
:0637E6008D28AB07AA06C6
:1037EC00908002E030E5079065787403F022906ACF
:1037FC0076E0FCA3E0FDA3E0FEA3E0F52C8E2B8D80
:10380C002A8C29AE02AF038E838F8263A201E52B33
:10381C00540744D0F583852C8263A201AF28122370
:10382C002AE4FCFDFEE52C2528F52CEE352BF52B9A
:10383C00ED352AF52AEC3529F529908058E529F043
:10384C00A3E52AF0A3E52BF0A3E52CF090800274FD
:10385C0020F0AF2CAE2BAD2AAC29906A76121EAAA2
:01386C002239
:0234F7008F281C
:1034F900908001E030E5099065787402F07F002240
:10350900906A7AE0FCA3E0FDA3E0FEA3E0F52C8E2F
:103519002B8D2A8C2990667B63A201E52B540744E5
:10352900C8F583852C8263A2017F06122340E52C0E
:103539002406F52CE4352BF52BE4352AF52AE43558
:1035490029F52990657963A201E52B540744C8F54B
:1035590083852C8263A201AF28122340E4FCFDFE7F
:10356900E52C2528F52CEE352BF52BED352AF52AFA
:10357900EC3529F52990804CE529F0A3E52AF0A33B
:10358900E52BF0A3E52CF09080017420F0AF2CAE70
:0D3599002BAD2AAC29906A7A121EAAAF2829
:0135A6002202
:102FD0009081E0E0F5280528052805280528052822
:102FE00005280528052805280528908010E0F52BE0
:102FF000A3E0F52CA3E0F52DA3E0F52E9081E1E010
:10300000F528052805280528052805280528052868
:10301000052805280528908014E0F52FA3E0F53059
:10302000A3E0F531A3E0F532E531B52D08E532B581
:103030002E037F0022E4F528E531540744E0F583B0
:1030400085328263A20190637563A2017F08122317
:103050007090637763A2019062AE63A2017F061253
:1030600022B8906375E0F529A3E0F52AE4F52890ED
:103070006375E0702AA3E024F8F528E5315407448D
:10308000E0F58385328274082582F582E43583F584
:103090008363A20190637563A201AF28122370AE0F
:1030A00029E4FCFDE532252AF532E5313EF531ED26
:1030B0003530F530EC352FF52F908014E52FF0A347
:1030C000E530F0A3E531F0A3E532F09080007440E4
:0330D000F0AF2836
:0130D30022DA
:10256A009081E6E0F528052805280528052805288C
:10257A0005280528052805280528908028E0F52B38
:10258A00A3E0F52CA3E0F52DA3E0F52E9081E7E07A
:10259A00F5280528052805280528052805280528D9
:1025AA0005280528052890802CE0F52FA3E0F530B2
:1025BA00A3E0F531A3E0F532E4F528E531B52D0ABB
:1025CA00E532B52E05C2200226D6E531540744F07D
:1025DA00F58385328263A20190637563A2017F0845
:1025EA00122370906375E0F529A3E0F52AE52A45E0
:1025FA002970099080027410F07F0022906682E0B0
:10260A00FFF46030906377E06F600302269D906666
:10261A0083E0FF906378E06F7079906684E0FF90C2
:10262A006379E06F706D906685E0FF90637AE06F82
:10263A006031805F906377E0906682F0906378E023
:10264A00906683F0906379E0906684F090637AE014
:10265A00906685F090637BE0FFA3E0906349CFF03A
:10266A00A3EFF0906375E0702AA3E024F8F528E55B
:10267A0031540744F0F58385328274082582F58245
:10268A00E43583F58363A20190637563A201AF28E1
:10269A00122370AE29E4FCFDE532252AF532E53134
:1026AA003EF531ED3530F530EC352FF52FAF2EAE46
:1026BA002DAD2CAC2BAB32AA31A930A82FD3121EC8
:1026CA009940099080027410F07F002290802CE5D6
:1026DA002FF0A3E530F0A3E531F0A3E532F09080C6
:0626EA00027440F0AF286D
:0126F00022C7
:1029DE009081E3E0F5280528052805280528052817
:1029EE000528052805280528052890801CE0F52BCC
:1029FE00A3E0F52CA3E0F52DA3E0F52E9081E4E005
:102A0E00F528052805280528052805280528052860
:102A1E00052805280528908020E0F52FA3E0F53045
:102A2E00A3E0F531A3E0F532E4F528E531B52D0A42
:102A3E00E532B52E05C221022B29E531540744E8B3
:102A4E00F58385328263A20190600463A2017F0E3A
:102A5E00122386906004E0F529A3E0F52A90600C1D
:102A6E00E0FFF4604590667BE0FEEF6E706EA3E0D3
:102A7E00FF90600DE06F706490667DE0FF90600ED9
:102A8E00E06F705890667EE0FF90600FE06F704CC4
:102A9E0090667FE0FF906010E06F7040906680E07F
:102AAE00FF906011E06F60048032D2D9906004E034
:102ABE00702AA3E024F2F528E531540744E8F583A3
:102ACE00853282740E2582F582E43583F58363A206
:102ADE000190600463A201AF28122386AE29E4FCA4
:102AEE00FDE532252AF532E5313EF531ED3530F58D
:102AFE0030EC352FF52FAF2EAE2DAD2CAC2BAB32DF
:102B0E00AA31A930A82FD3121E995006E52A4529BD
:102B1E0070099080017410F07F0022908020E52FC4
:102B2E00F0A3E530F0A3E531F0A3E532F09080019B
:052B3E007440F0AF2817
:012B4300226F
:0430D4008E2D8F2E80
:1030D800908000E030E5079065787401F022906AEE
:1030E80072E0FCA3E0FDA3E0FEA3E0F5348E338D8F
:1030F800328C31E534FFE5335407FEE42FF530EE2A
:1031080034C0F52F853082F5837423F00530E5301F
:103118007002052F532FC7F582852F83740AF00597
:1031280030E5307002052F532FC790633E63A2012C
:10313800852F8385308263A2017F0612232A7406B5
:103148002530F530E4352FF52F852D83852E8263C4
:10315800A201852F8385308263A20112230EE4FC2D
:10316800FDFE906A72E0F8A3E0F9A3E0FAA3E02F6D
:10317800FFEE3AFEED39FDEC38FCEF2408FFE43EA3
:10318800FEE43DFDE43CFC906A72121EAA906A724D
:10319800E0908040F0906A73E0908041F0906A740B
:1031A800E0908042F0906A75E0908043F090800053
:0331B8007420F090
:0131BB0022F1
:0A2EC9008E2D8F2E8C2F8D308B3153
:102ED300908000E030E5079065787401F022906AF5
:102EE30072E0FCA3E0FDA3E0FEA3E0F5378E368D90
:102EF300358C34E537FFE5365407FEE42FF533EE22
:102F030034C0F532853382F5837423F00533E5331A
:102F1300700205325332C7F582853283740AF00595
:102F230033E533700205325332C790633E63A20127
:102F330085328385338263A2017F0612232A7406B6
:102F43002533F533E43532F532852D83852E8263BF
:102F5300A20185328385338263A20112230E8F3847
:102F6300EF2533F533E43532F532E5316017852F3C
:102F73008385308263A20185328385338263A20114
:102F8300AF3112232AE53824082531F531FFE4FC5B
:102F9300FDFEE5372FF537EE3536F536ED3535F5EC
:102FA30035EC3534F534908040E534F0A3E535F065
:102FB300A3E536F0A3E537F09080007420F0AF3737
:0C2FC300AE36AD35AC34906A72121EAA16
:012FCF0022DF
:06329D008E288F298D2A06
:1032A300908000E030E5079065787401F022906A21
:1032B30072E0FCA3E0FDA3E0FEA3E0F5308E2F8DCA
:1032C3002E8C2DE530FFE52F5407FEE42FF52CEE71
:1032D30034C0F52B852C82F5837423F0052CE52C63
:1032E3007002052B532BC7F582852B83EBF0052C3E
:1032F300E52C7002052B532BC790633E63A2018517
:103303002B83852C8263A2017F0612232A74062550
:103313002CF52CE4352BF52B85288385298263A294
:1033230001852B83852C8263A201AF2A12232A7481
:1033330008252AF52AFFE4FCFDFEE5302FF530EEE3
:10334300352FF52FED352EF52EEC352DF52D9080FF
:1033530040E52DF0A3E52EF0A3E52FF0A3E530F033
:103363009080007420F0AF30AE2FAD2EAC2D906A5C
:0433730072121EAA0A
:013377002233
:0238F2008F4104
:1038F400908000E030E5079065787401F022906ACA
:1039040072E0FCA3E0FDA3E0FEA3E0F5458E448D48
:10391400438C42E545FFE5445407FEE42FFFEE34B3
:10392400C09062B463A201F5838F8263A201AF41A8
:1039340012232AE4FCFDFEE5452541F545EE354418
:10394400F544ED3543F543EC3542F542908040E5CE
:1039540042F0A3E543F0A3E544F0A3E545F09080ED
:10396400007420F0AF45AE44AD43AC42906A72128D
:023974001EAA89
:01397600222E
:0631BC008E288F29AB05EF
:1031C200908000E030E5079065787401F022906A03
:1031D20072E0FCA3E0FDA3E0FEA3E0F52F8E2E8DAE
:1031E2002D8C2CE52FFFE52E5407FEE42FF52BEE58
:1031F20034C0F52A852B82F5837423F0052BE52B49
:103202007002052A532AC7F582852A83EBF0052B23
:10321200E52B7002052A90633E63A201852A83850D
:103222002B8263A2017F0612232A7406252BF52B1B
:10323200E4352AF52A532AC7E528852B82852A8375
:10324200F0052BE52B7002052A532AC7F582852A41
:1032520083E529F0052BE52B7002052A532AC7E5E1
:103262002F240AF52FE4352EF52EE4352DF52DE425
:10327200352CF52C908040E52CF0A3E52DF0A3E54C
:103282002EF0A3E52FF09080007420F0AF2FAE2E29
:0A329200AD2DAC2C906A72121EAA3A
:01329C00220F
:1035A700E4F528E5282401FFE433FE123DD87436FC
:1035B7002528F582E43463F583EFF00528E528C371
:1035C700943F40DFE4F528E528247FFFE433FE122B
:1035D7003DD8742D2528F582E43461F583EFF07426
:1035E7002D2528F582E43461F583E0FF6003B4FFFD
:1035F7001D742D2528F582E43461F5837420F07459
:103607002E2528F582E43461F583E4F08009052846
:10361700E528C3948040B0E49061ACF0F528AF286A
:103627007E00123DD874AD2528F582E43461F58318
:0B363700EFF00528E528C394FE40E3F7
:013642002265
:10405600E4FDFCC3ED9FEC9E5015E4FBFA0BBB00A0
:0F406600010ABA01F8BB90F50DBD00010C80E412
:014075002228
:0D4136004390014390025390FE5390FD22F0
:0D4143005390FD5390FE43900243900122E3
:0E4127005390FD439002E5905408FF5390FD25
:014135002267
:0D4150005390FD4390014390025390FD22D7
:07416800AE071FEE70FA2202
:023F6900AD07A2
:103F6B00E4FC5390FDEDA804088002C333D8FC3069
:103F7B00E70543900180035390FE7F051241684390
:093F8B0090020CBC08DC5390FD0F
:013F9400220A
:103FBF00E4FF5390FD7E07439002E59030E00D74CF
:103FCF0001A806088002C333D8FC42075390FD1E98
:083FDF00C3EE6480948050DF02
:013FE70022B7
:103F9500AB05AA071241367FA0123F69124127AF30
:103FA50002123F69124127AF03123F6912412712DE
:0A3FB50041437F0A7E0012405622AD
:043DD800AB07AA0685
:103DDC00C3EB94FFEA9400400DE42BF58274773A20
:103DEC00F583E493FF221241367FA0123F69124102
:103DFC0027AF03123F691241271241367FA1123FB0
:0D3E0C0069124127123FBF1241501241437D
:013E19002286
:023F03008B2D04
:103F0500A2AF9228C2AF85A22E53A2FE8E838F82C6
:103F150005A28C838D8274091223B4E52D53A2FE6C
:103F250043A2201223B653A2DF852EA2A22892AF68
:013F3500FF8C
:013F36002268
:10409400A2AF9228C2AF8C838D82EF1223B443A2C5
:0C40A400201223B653A2DFA22892AFFF27
:0140B00022ED
:02400E008F28F9
:10401000A2AF9228C2AFE4F5838D8274061223B456
:10402000E52843A2201223B653A2DFA22892AF7F35
:01403000018E
:01403100226C
:024032008F28D5
:10403400A2AF9228C2AFE4F5838D82740A1223B42E
:10404400E52843A2201223B653A2DFA22892AF7F11
:01405400016A
:014055002248
:1021DD00A907E7FFA805EF93C3966008403B74FC81
:1021ED002FFF80F00F08EF93C3966008402B74FB10
:1021FD002FFF80E00F08EF93C3966008401B74FA21
:10220D002FFF80D00F08EF93D3966008400B74F921
:10221D002FFF80C01F1F1F1F1FEF54FEF80303F772
:10222D00E893FC08E893FD08E893FE08E893FF2285
:10223D0009E993C39D6008402974FB29F980F109D0
:10224D00E993C39E6008401A74FA29F980E209E9FE
:10225D0093D39F6008400B74F929F980D31919198C
:10226D001919E9C313C313FF22740093F8ECC39833
:10227D004024701F740193F8EDC3984019701474C5
:0E228D000293F8EEC398400E7009740393F8A4
:10229B00EFC39840037F00227F0122EDF8E6F008A0
:1022AB00A3DFFA22EDF8E0F608A3DFFA22E0A3633E
:1022BB00A201F0A363A201DFF475A2002263A201C5
:1022CB00F0A363A20122E0A363A201F0A363A20126
:1022DB00E0A363A201F0A363A201E463A201F0A354
:1022EB0063A201DFE175A20022E0A363A2016DFEF0
:1022FB00936CFDEE058393FC158363A201DFEA75F6
:10230B00A200227F00E493A363A201F00F600CA351
:10231B00E583C2E3F58363A20180EA75A20022E0A4
:10232B00A363A201F0A3E583C2E3F58363A201DFFC
:10233B00EE75A20022E0A363A201F0A3E583C2E441
:10234B00D2E3F58363A201DFEC75A20022E0A36365
:10235B00A201F0A3E58344F8C2E5F58363A201DF94
:10236B00EC75A20022E583C2E3F583E0A363A2012F
:10237B00F0A363A201DFEE75A20022E583C2E4D2D3
:0A238B00E3F583E0A363A201F0A3D1
:1023950063A201DFEC75A20022E58344F8F583E032
:1023A500A363A201F0A363A201DFEE75A20022F9E7
:1023B50022C002C004C00612FFF0D006D004D0022D
:0123C50022F5
:100E280042415544004E4F5F4D45414E4452005794
:100E38005F4D4F44454D00534C415645004C45418C
:100E480044455200494E565F52454300494E565F4D
:100E58005452414E5300494E565F414C4C004B5042
:100E68000054555F5155414E004D41470054495477
:100E7800524551005453524551004752414E49542E
:100E88005F4F4C4400475400000A53656E643A2093
:100E9800000A435243206572726F722120000A5281
:100EA8006563204F4B2120003E2A2C312CCFE0F0E7
:100EB800E0ECE5F2F0FB20F1E8EDF5F0EEEDEDEE1B
:100EC800E3EE20EFEEF0F2E00A003E4C2C42303127
:100ED8002C256C752CD1EAEEF0EEF1F2FC20EEE157
:100EE800ECE5EDE02C35302C3130302C3230302C24
:100EF8003330302C3630302C313230302C323430E4
:100F0800302C343830300A003E422C4731302C2502
:100F180062752CC8EDE2E5F0F1E8FF20EDE020EF86
:100F2800F0E8B8ECE50A003E422C4731312C256246
:100F3800752CC8EDE2E5F0F1E8FF20EDE020EFE5E3
:100F4800F0E5E4E0F7E50A003E422C4730322C2574
:100F580062752CD3EFF0E0E2EBE5EDE8E520EFEE8B
:100F6800F2EEEAEEEC2020285254532D4354532934
:100F78000A003E532C4730332C256C752CC7E0E40F
:100F8800E5F0E6EAE020F1F2E0F0F2E020EFE5F04B
:100F9800E5E4E0F7E828ECF1290A003E532C473055
:100FA800332C256C752C202AE7E0E4E5F0E6EAE02E
:100FB80020F1F2E0F0F2E020EFE5F0E5E4E0F7E818
:100FC80028ECF1290A003E2A2C312CC0E4E0EFF28B
:100FD800E5F020F1E8EDF5F0EEEDEDEEE3EE20EAD8
:100FE800E0EDE0EBE02E20CFF0EEF2EEEAEEEB20C3
:100FF80022C3F0E0EDE8F2220A003E422C473132EB
:101008002C2562752CC7E0EFF0E5F220E3E5EDE56D
:10101800F0E0F6E8E820ECE5E0EDE4F0E00A003E78
:10102800422C4731332C2562752CD0E5E6E8EC20BC
:1010380022E2E5E4EEECFBE9220A003E422C4731CD
:10104800342C2562752C2B20ECE5E0EDE4F020EF44
:10105800E5F0E5E420EEF2EAF0FBE2E0FEF9E8EC88
:1010680020F4EBE0E3EEEC0A003C21003C42303196
:101078003D003C4731303D003C4731313D003C4765
:1010880030323D003C4730333D003C4731323D0073
:101098003C4731333D003C4731343D00FF0E28FFCB
:1010A8000E2DFF0E37FF0E3FFF0E45FF0E4CFF0EB5
:1010B80054FF0E5EFF0E66FF0E69FF0E71FF0E7580
:1010C800FF0E7CFF0E82FF0E8DFF0E900008040CB1
:1010D800020A060E0109050D030B070F0011233242
:1010E800465765748C9DAFBECADBE9F81001332200
:1010F800564775649C8DBFAEDACBF9E821300213F0
:1011080067764455ADBC8E9FEBFAC8D931201203DF
:1011180077665445BDAC9E8FFBEAD8C942536170CF
:1011280004152736CEDFEDFC8899ABBA52437160BF
:1011380014053726DECFFDEC9889BBAA63724051AF
:1011480025340617EFFECCDDA9B88A9B736250419F
:1011580035241607FFEEDCCDB9A89A8B8495A7B67F
:10116800C2D3E1F008192B3A4E5F6D7C9485B7A67F
:10117800D2C3F1E018093B2A5E4F7D6CA5B486976F
:10118800E3F2C0D129380A1B6F7E4C5DB5A496875F
:10119800F3E2D0C139281A0B7F6E5C4DC6D7E5F44F
:1011A8008091A3B24A5B69780C1D2F3ED6C7F5E43F
:1011B8009081B3A25A4B79681C0D3F2EE7F6C4D52F
:1011C800A1B082936B7A48592D3C0E1FF7E6D4C51F
:1011D800B1A092837B6A58493D2C1E0F0089129B4F
:1011E80024AD36BF48C15AD36CE57EF78108931AFF
:1011F800A52CB73EC940DB52ED64FF76028B1099EF
:1012080026AF34BD4AC358D16EE77CF5830A9118DE
:10121800A72EB53CCB42D950EF66FD74048D169FBE
:1012280020A932BB4CC55ED768E17AF3850C971EBE
:10123800A128B33ACD44DF56E960FB72068F149DAE
:1012480022AB30B94EC75CD56AE378F1870E951C9E
:10125800A32AB138CF46DD54EB62F97008811A939E
:101268002CA53EB740C952DB64ED76FF89009B127E
:10127800AD24BF36C148D35AE56CF77E0A8318916E
:101288002EA73CB542CB50D966EF74FD8B0299105E
:10129800AF26BD34C34AD158E76EF57C0C851E973E
:1012A80028A13AB344CD56DF60E972FB8D049F163E
:1012B800A920BB32C54CD75EE168F37A0E871C952E
:1012C8002AA338B146CF54DD62EB70F98F069D141E
:0C12D800AB22B930C74ED55CE36AF17858
:1040B70052668D00000000000000000000000000B4
:0540C7000000000000F4
:10407600906A67E06FFC9011E493FE906A66E06ECA
:0D408600A3F0AF04EF9010E493906A66F091
:01409300220A
:0100320022AB
:103B5D00906A68E02424F582E43468F5837420F0DB
:103B6D00906A68E004F0E4906A86F0906A86E0FE60
:103B7D00C39D503FEF75F003A424A4F582E43410E7
:103B8D00F583E493FB740193FA740293F98E8275B5
:103B9D008300121D7EFE906A68E02424F582E434D1
:103BAD0068F583EEF0906A86E004F0906A68E004B0
:033BBD00F080B8DD
:013BC00022E2
:103ECD00906A86EFF0906A86E0242DF582E43461E5
:103EDD00F583E0FF6420601D906A68E02424F5827C
:103EED00E43468F583EFF0906A86E004F0906A6838
:053EFD00E004F080D09C
:013F0200229C
:101A8600E4906A68F0906A7EF0906A7EE075F003F2
:101A9600A424A4F582E43410F583E493FB74019343
:101AA600FA740293F9121D657003021D64E4906ACC
:101AB60080F0A3F0906A7FF0906A7FE0242DF58293
:101AC600E43461F583E0FF7003021D5B906A7EE0FB
:101AD60075F003A424A4F582E43410F583E493FBA3
:101AE600740193FA740293F9906A80E0F582758323
:101AF60000121D7EFEEFB5060F906A817401F0900C
:101B06006A80E004F0021D52906A81E07003021DB3
:101B160052EE6003021D49906A7EE0FF906A80E003
:101B2600FD123B5D906A7EE0B40F004003021D5B30
:101B3600901B3DF8282873021B6A021C24021C29EC
:101B4600021C64021C69021C6E021C73021C7802D1
:101B56001C7F021CBA021CF2021CF6021CFA021CB2
:101B6600FE021D02906A7FE0FF123ECD906A7FE082
:101B7600242DF9E43461FA7B01C0031B8B2B752CF1
:101B860000752D00E4F52ED0031223C6906A82124A
:101B96001EAAE4FFFEFDFC906A82E0F8A3E0F9A32A
:101BA600E0FAA3E0FBC3121E996028906A82E0F86F
:101BB600A3E0F9A3E0FAA3E0FBE47F207E1CFDFC92
:101BC600121DF9121E8B906A6CEEF0A3EFF0E490F2
:101BD6006A6BF0E47FB07E04FDFC906A82E0F8A3B5
:101BE600E0F9A3E0FAA3E0FBD3121E995003021D0D
:101BF6005B906A6B7401F0906A82E0F8A3E0F9A347
:101C0600E0FAA3E0FB7F007EC27D017C00121DF995
:101C1600121E8B906A6CEEF0A3EFF0021D5BD204ED
:101C2600021D5B906A7FE0FF123ECDD213906A7F61
:101C3600E0242DF9E43461FA7B01C0031B8B2B757C
:101C46002C00752D00E4F52ED0031223C6906A826F
:101C5600121EAA906A85E090669FF0021D5BD2175D
:101C6600021D5BD211021D5BD20E021D5BD20B025E
:101C76001D5BD20ED20B021D5B906A7FE0FF123E07
:101C8600CD906A7FE0242DF9E43461FA7B01C0032C
:101C96001B8B2B752C00752D00E4F52ED00312231B
:101CA600C6906A82121EAA906A85E0547F906A6A7C
:101CB600F0021D5B906A7FE0FF123ECD906A7FE0E6
:101CC600242DF9E43461FA7B01C0031B8B2B752CA0
:101CD60000752D00E4F52ED0031223C6906A8212F9
:101CE6001EAA906A85E09067A3F08069D206806597
:101CF600D20D8061D20C805DC20A8059906A7FE065
:101D0600FF123ECD906A7FE0242DF9E43461FA7B20
:101D160001C0031B8B2B752C00752D00E4F52ED00E
:101D2600031223C6906A82121EAA906A84E0FEA35A
:101D3600E0FF7C007D06121DAB9066A0EEF0A3EFDF
:101D4600F08012E4906A81F0906A80F0906A7FE0F9
:0E1D560004F0021ABE906A7EE004F0021A8FBA
:011D6400225C
:10001E00EF540F9010D493FEC454F0FEEFC4540F5F
:04002E00932EFF22EC
:103F370030162CE4906475F0E51C24FEFFA3F09086
:103F4700667AE0906477F0A37408F090696663A2DC
:103F57000190647963A2011222B8C2167F01227F01
:023F6700002236
:103D38008F1EC228E4FFE51B64056033E51EB47ED0
:103D480005D205A22822E51E30E707431001051B0E
:103D580080065310FEE4F51B0517E517B40808851F
:103D68001018D228E4F517E51025E0F510800DE5C8
:103D78001E30E705D205A22822E4F51BE51E25E042
:083D8800F51E0FBF08B0A228D0
:013D90002210
:103AEF00E4FEE51625E0F516EF30E7364316012024
:103AFF0028330515E515B4052CE4F515051AE51A57
:103B0F00B408170514E514AC137002051314F582ED
:103B1F008C83E516F0051DE4F51AE51625E0F5167C
:103B2F008003E4F515051AE51AB408170514E51412
:103B3F00AC137002051314F5828C83E516F0051D86
:0D3B4F00E4F51AEF25E0FF0EEE6408709516
:013B5C002246
:103FE800906A6C74FFF0A374B8F0E4906A6BF09078
:103FF8006A6A04F0E4906A68F012286CEF600312B1
:064008001A86123C24227E
:1040CD0075657E7562A0C208D210C216D231C214B7
:0C40DD00C202C215D201C212123E5C22C7
:042DB4008E298F2AAB
:102DB800906A66E0906A80F0906A67E0906A81F0B5
:102DC800E4F51DF515906A66F0A3F0AB2AAA2975FB
:102DD80013697514E63011258514828513837405EB
:102DE800F00514E51470020513F5828513837455F4
:102DF800F00514E51470020513051D051D851482E0
:102E0800851383747EF00514E51470020513051DFF
:102E1800E4F51A906A7EF0906A7EE0C39D50498B73
:102E2800828A83E0FF12001E906A7FEFF0906A6743
:102E3800E06F906A7FF0E0FF9011E493FE906A667D
:102E4800E06EA3F0EF9010E493906A66F00BEBAE9F
:102E58000270010A14F5828E83E0FFC228123AEF4D
:102E6800906A7EE004F080AF906A67E0FF12001E6F
:102E7800C228123AEF906A66E0FF12001EC22812BA
:102E88003AEFD2287F7E123AEFD228E4FF123AEFC7
:102E9800201307D228E4FF123AEFD2027C697DE6BC
:102EA8008C138D143025097E0E7F91AB1D122EC90F
:102EB800906A80E0906A66F0906A81E0906A67F0B4
:012EC80022E7
:103E1A008F2820022030120E7E697F26E52824FC96
:103E2A00FD122DB4800C7E637F79E52824FCFD12F7
:103E3A002DB4C21222201219852819D21290637940
:103E4A0063A20190692663A201E52824FCFF1222DD
:023E5A00B8228C
:10344200E4FF0F2405F582E43461F5837408F00F7C
:1034520074052401F582E43461F583E4F07C667D31
:1034620092FEED1DAA0470011CF5828A83E0FBAA7C
:10347200070F74052AF582E43461F583EBF00EBE82
:1034820004E07C667D96E4FEED1DAA0470011CF545
:10349200828A83E0FBAA070F74052AF582E434616D
:1034A200F583EBF00EBE04E07C667D9AE4FEED1D32
:1034B200AA0470011CF5828A83E0FBAA070F740537
:1034C2002AF582E43461F583EBF00EBE04E07C66FB
:1034D2007D9EE4FEED1DAA0470011CF5828A83E044
:1034E200FBAA070F74052AF582E43461F583EBF039
:0434F2000EBE04E026
:0134F60022B3
:102B4400200803022C4FE5605438655B7003022CA7
:102B54009CE55B24085438F55B131313541F244B72
:102B6400F8E6F51820053020072DFF123D3850D621
:102B7400AF1812001E1240760512E512AE11700253
:102B8400051114F5828E83E518F0051CE51CD39419
:102B94008040B3D20780AFE51CD394024002D21622
:102BA400C208C205E4F549D231906966E070052097
:102BB4000702D203C207906A67E0FF906A66E04F9B
:102BC400604CC21630250D7E0E7F997C697D66AB04
:102BD4001C122EC9906697E0FCA3E0FDA3E0FEA3BF
:102BE400E0FFE4FAF9F8EF2401FFEA3EFEE93DFDD7
:102BF400E83CFC906697121EAA906A69E004F0D340
:102C040094055003022B4AD203E4F0022B4A3025E8
:102C14000D7E0E7FA67C697D66AB1C122EC9906664
:102C24008FE0FCA3E0FDA3E0FEA3E0FFE4FAF9F8E3
:102C3400EF2401FFEA3EFEE93DFDE83CFC90668F8F
:102C4400121EAAE4906A69F0022B4A20314AE54B2D
:102C5400647E7024300307F549D231C20322D201C5
:102C6400D208E4F51CF51B906A67F0906A66F0F5EB
:102C74001775116975126622E54BB4A01620061368
:102C8400D2019066A0E0FFA3E0906924CFF0A3EF07
:092C9400F0C209E4F549D2312235
:101FE800300F2DC3E5489564FFE5479563FED3EFB1
:101FF8009440EE940040197B087D40AF64AE6312B4
:10200800329DE5642440FFE43563540FF5638F6423
:10201800201B030221DC301A0AC21A9067A2E06072
:102028000214F0301003122B442014030220B8E5E8
:1020380061655C6048E56124085438FFE55C543804
:102048006F60047E0180027E00E51D60047D0180D2
:10205800027D00EE5D70030221DC0514E514AC136B
:102068007002051314F5828C83E0FEE561131313E7
:10207800541F2453F8A6068F61151D80B8C214C2D8
:1020880002906693E0FCA3E0FDA3E0FEA3E0FFE47A
:10209800FAF9F8EF2401FFEA3EFEE93DFDE83CFCD1
:1020A800906693121EAAD215D2B1E49067A2F022CC
:1020B8003008030221DC30024FE561655C600302F1
:1020C80021DC30B10AC2B190669FE09067A2F0307F
:1020D800130C30B0099067A2E060030221DC0514FC
:1020E800E514AE137002051314F5828E83E0FFE544
:1020F80061131313541F2453F8A607E561240854E9
:1021080038F561151DD21422301206AF19123E1A85
:1021180022E561655C60030221DC3004030221DCF6
:1021280030B10AC2B190669FE09067A2F030130CFC
:1021380030B0099067A2E060030221DC20012590FD
:10214800669BE0FCA3E0FDA3E0FEA3E0FFE4FAF950
:10215800F8EF2401FFEA3EFEE93DFDE83CFC90660D
:102168009B121EAAC201E561131313541F2453F8CE
:1021780076AAE56124085438F561131313541F2413
:1021880053F876A0E56124085438F5611313135405
:102198001F2453F8E4F6E56124085438F561131355
:1021A80013541F2453F8E4F6E56124085438F56104
:1021B800131313541F2453F8E4F6E5612408543824
:1021C800F561131313541F2453F8E4F6E56124084A
:0521D8005438F56122FE
:0B415D00301505C2157F01227F0022F3
:102C9D007BFF7A0E79B012178C906A6BE06033A3CC
:102CAD00E0FEA3E0FFC3E49FFFE49EFEAB07FA3313
:102CBD0095E0F9F87F007EC27D017C00121DF98F31
:102CCD00338E328D318C307BFF7A0E79D212178C88
:102CDD008032906A6CE0FEA3E0FFC3E49FFFE49EA8
:102CED00FEAB07FA3395E0F9F8E47F207E1CFDFC7E
:102CFD00121DF98F338E328D318C307BFF7A0E7928
:102D0D00D212178C7BFF7A0F7910A20EE433F530B7
:102D1D0012178C7BFF7A0F792FA20BE433F530124B
:102D2D00178C7BFF7A0F7950A213E433F53012170D
:102D3D008C30131F7BFF7A0F797A90669FE075F0C8
:102D4D000AA4FFAEF0E48F338E32F531F530121751
:102D5D008C801D7BFF7A0F79A390669FE075F00A3A
:102D6D00A4FFAEF0E48F338E32F531F53012178CAF
:102D7D007BFF7A0F79CE12178C7BFF7A107902A226
:102D8D0004E433F53012178C7BFF7A107927A217E4
:102D9D00E433F53012178C7BFF7A107943A211E4DE
:072DAD0033F53012178C22F0
:10286C007E107F7112386DEF4E70037F01227E1047
:10287C007F7412386DEF4E7003022913123C829054
:10288C006A7E121EAAE4FFFEFDFC906A7EE0F8A3AD
:10289C00E0F9A3E0FAA3E0FBC3121E996025906A4D
:1028AC007EE0F8A3E0A3E0A3E0E47F207E1CFDFC27
:1028BC00121DF9121E8B906A6CEEF0A3EFF0E490EF
:1028CC006A6BF0E47FB07E04FDFC906A7EE0F8A3B6
:1028DC00E0F9A3E0FAA3E0FBD3121E994038906A0A
:1028EC006B7401F0906A7EE0F8A3E0A3E0A3E07FB4
:1028FC00007EC27D017C00121DF9121E8B906A6C49
:10290C00EEF0A3EFF0800F906A6C74FFF0A374B834
:10291C00F0E4906A6BF07E107F7A12386DEF4E60A7
:10292C000C1240E9EF24D024FF920E8002C20E7EDE
:10293C00107F8012386DEF4E600C1240E9EF24D0FE
:10294C0024FF920B8002C20B7E107F8612386DEF33
:10295C004E600C1240E9EF24D024FF92138002C287
:10296C00137E107F8C12386DEF4E6013123C82E494
:10297C007B0AFAF9F8121DF990669FEFF08005E4D6
:10298C0090669FF07E107F9212386DEF4E600C12A5
:10299C0040E9EF24D024FF92048002C2047E107F11
:1029AC009812386DEF4E600C1240E9EF24D024FFE2
:1029BC0092178002C2177E107F9E12386DEF4E6008
:1029CC000C1240E9EF24D024FF92118002C2117F37
:0129DC0000FA
:0129DD0022D7
:03416F00C2AE22BB
:10410300BF360BD20FE4F547F548F563F564BF37C7
:0441130002C20F22B3
:103C2400C2A9438902906A6DE0FFF58C8F8A75D929
:103C34000475DA4875DB3175DC4975DD4975DE31AB
:103C4400E4F5E9F5F9F5EBF5FB906A6BE0601675C0
:103C5400EC1075ED10E4F5FCF5FD755F08755D106D
:103C6400755E01801375EC8075ED80E4F5FCF5FD5F
:0E3C7400755F80F55D755E10E4F5EEF5FE22DD
:103E5C00E4FEAF8CEFFD906A6CE07003A3E06D6044
:103E6C0005123C247E01E5D920E2057E02123C2499
:103E7C00E58920E105123C247E03D28C75D840756F
:083E8C00B740D2AED2AFAF0681
:013E9400220B
:030033000226F1B1
:0B26F100C0E0C083C082C0D075D008DC
:1026FC00C2AF30DC56C3E5EC95EEC3955F5012E5E6
:10270C005E25ECF5EC30D70405FC801685FCFC80CE
:10271C0011C3E5EC955EF5EC30D70415FC80038510
:10272C00FCFC300F24854882854783E590F00548F2
:10273C00E54870020547F582854783E5EEF00548CC
:10274C00E5487002054753470FC2DC30D929300FDA
:10275C0024854882854783E590F00548E54870025A
:10276C000547F582854783E5EBF00548E54870029F
:10277C00054753470FC2D930DA67E55D700405FC95
:10278C008010E55D25ECF5EC30D70405FC80038565
:10279C00FCFCE5495480F546E54925E0F5493097C0
:1027AC00020549200E03634901303119E54965657D
:1027BC006006E54965627027755B007560008549A8
:1027CC004BC231801A0560E5605407701253603FAC
:1027DC00E560131313541F244BF8A649754900C226
:1027EC00DA30DB71E55D700405FD8010E55D25EDEB
:1027FC00F5ED30D70405FD800385FDFDE561655CD5
:10280C006029E55C54077013E55C131313541F2403
:10281C0053F8E6F54A200B03634AFFE54A339296D8
:10282C00E54A25E0F54A055C535C3FB292300F2334
:10283C00854882854783E590F00548E54870020598
:10284C0047F582854783E4F00548E5487002054763
:07285C0053470FC2DBD2AFAE
:09286300D0D0D082D083D0E03245
:1036DF0002085FE493A3F8E493A34003F68001F29A
:1036EF0008DFF48029E493A3F85407240CC8C333EC
:1036FF00C4540F4420C8834004F456800146F6DFBB
:10370F00E4800B01020408102040809040B1E47E59
:10371F00019360BCA3FF543F30E509541FFEE493AF
:10372F00A360010ECF54C025E060A840B8E493A376
:10373F00FAE493A3F8E493A3C8C582C8CAC583CAA1
:10374F00F0A3C8C582C8CAC583CADFE9DEE780BE59
:0140CC0000F3
:101D6500BB010689828A83E0225002E722BBFE027C
:091D7500E32289828A83E49322AF
:101D7E00BB010CE58229F582E5833AF583E022501A
:101D8E0006E92582F8E622BBFE06E92582F8E22264
:0D1D9E00E58229F582E5833AF583E493227E
:101DAB00EF8DF0A4A8F0CF8CF0A428CE8DF0A42E4C
:021DBB00FE2206
:101DBD0075F008758200EF2FFFEE33FECD33CDCCDD
:101DCD0033CCC58233C5829BED9AEC99E582984060
:101DDD000CF582EE9BFEED9AFDEC99FC0FD5F0D63D
:101DED00E4CEFBE4CDFAE4CCF9A88222B800C1B967
:101DFD000059BA002DEC8BF084CFCECDFCE5F0CBA5
:101E0D00F97818EF2FFFEE33FEED33FDEC33FCEBDD
:101E1D0033FB10D703994004EB99FB0FD8E5E4F998
:101E2D00FA227818EF2FFFEE33FEED33FDEC33FC85
:101E3D00C933C910D7059BE99A4007EC9BFCE99A79
:101E4D00F90FD8E0E4C9FAE4CCFB2275F010EF2FBE
:101E5D00FFEE33FEED33FDCC33CCC833C810D707BE
:101E6D009BEC9AE899400AED9BFDEC9AFCE899F8F9
:0E1E7D000FD5F0DAE4CDFBE4CCFAE4C8F9228C
:0E1E8B00C3E49FFFE49EFEE49DFDE49CFC2268
:101E9900EB9FF5F0EA9E42F0E99D42F0E89C45F09F
:011EA9002216
:0C1EAA00ECF0A3EDF0A3EEF0A3EFF022AB
:101EB600A8828583F0D083D082121ECD121ECD1249
:101EC6001ECD121ECDE473E493A3C583C5F0C5836E
:101ED600C8C582C8F0A3C583C5F0C583C8C582C876
:011EE60022D9
:10172A00E53C2430F8E6053C22782D302F0278304B
:10173A00E475F001121F48021D652028EB7F2ED2A6
:10174A00288018EF540F2490D43440D4FF302C0B47
:10175A00EF24BFB41A0050032461FFE53D6002156F
:10176A003D0540E5407002053F302F0D782DE475A8
:10177A00F001121F48EF021EE7023D917403D22FB7
:10178A008003E4C22FF53C8B2D8A2E892FE4F53D88
:10179A00F53FF540E53D60077F2012176580F57536
:1017AA003EFFC229C228C22AC22BC22DC22EC23073
:1017BA00121733FF700D302F057F00121776AF40D6
:1017CA00AE3F22B4255FC2D5C22C121733FF24D0F4
:1017DA00B40A00501A75F00A783D30D50508B6FFEC
:1017EA000106C6A426F620D5047002D22B80D9247D
:1017FA00CFB41A00EF5004C2E5D22C021976D229CE
:10180A0080C6D22880C0D22A80BCD2D580BAD22D36
:10181A0080B47F20121765202A077401B53D004065
:10182A00F112172AFF12176502179ED230D22E80A4
:10183A009512172AFB12172AFA12172AF94A4B701D
:10184A000679477A1A7BFF202A2EE53D602A7E0018
:10185A008E82758300121D7E60060EEE653E70F064
:10186A00C2D5EBC0E0EAC0E0E9C0E0EE1219BDD093
:10187A00E0F9D0E0FAD0E0FB121D65FF60AAEBC0E8
:10188A00E0EAC0E0E9C0E0121765D0E02401F9D02F
:10189A00E03400FAD0E0FBE53E0460DCD53ED980B6
:1018AA00877BFF7A1979B9D22A809C7910800279CC
:1018BA0008C22EC2308008D2D5790A8004790AC2B9
:1018CA00D5E53E047002F53EE4FAFDFEFF12172A42
:1018DA00FC7B0820291312172AFD7B1030280A12D4
:1018EA00172AFE12172AFF7B20EC3382D592D55095
:1018FA0013C3E43028069FFFE49EFEE42029039DDB
:10190A00FDE49CFCE4CBF8C229EC700CCFCECDCC24
:10191A00E824F8F870F38017C3EF33FFEE33FEEDD7
:10192A0033FDEC33FCEB33FB994002FB0FD8E9EBB8
:10193A00302905F8D0E0C448B229C0E00AEC4D4E7F
:10194A004F78207B0070C2EAB53E0040BCC0E0126E
:10195A0019BFD0F0D0E0202904C4C0E0C4B229C025
:10196A00F012174ED0F0D5F0EB02179E121FA718EF
:10197A003B5318B558180C4C18084218B94F18C1DF
:0F198A004418C14918214318C75518AB4618AB6C
:101999004518AB471A675018102D18142E18372BF5
:1019A9001818231835201A502A17D0480000182F64
:1019B9003F3F3F00790AA2D5202B14302D09B910D9
:1019C900020404B9080104A2D5202E025001042002
:1019D9002A68922AB53D005034C0E07F20302B1987
:1019E9007F30A22A722E722D500F121A16C22AC2E5
:1019F9002EC22DC2307F30800F302D03E9C0E01296
:101A09001765302D03D0E0F9D0E0B53DCC302D1766
:101A19007F30B9100C1217657F58302C077F7880FA
:101A290003B90803121765302A057F2D0217657F50
:101A3900202030F87F2B202EF322922A80CF286E87
:101A4900756C6C2900D22912172A3029F8C2297815
:101A59003D30D50108F60217D02D504349581217C9
:101A69002A2403B405004001E4901A629312175620
:0D1A7900743A121756D22B753D040218B5B1
:1023C6008B288A29892AE4F534F533F532F531F577
:1023D6002FF530E52C452D452B6012EBC0E0EAC009
:1023E600E0E9C0E0AB2BAA2CA92D121F58AB28059B
:1023F6002AE52AAA297002052914F9121D65F53560
:10240600C394094007E535D3940D40E1E5356420D2
:1024160060DBE535B42D054330038016E535B42B76
:1024260005433001800C74FF252AF52A74FF3529EF
:10243600F529E52E60046410703FAB28AA29A92A65
:10244600121D6564306009E52E702E752E0A8029EE
:10245600900001121D7EFF64786004EFB4581343A8
:102466003001752E107402252AF52AE43529F5293E
:102476008007E52E7003752E08AB28052AE52AAAE3
:10248600297002052914F9121D65F535C3946140BA
:102496000AE535D3947A50035335DF74D02535F5E4
:1024A60035C3940A400CE5359411406D74F9253511
:1024B600F535E535D3952E506043300185343985A1
:1024C6003338853237853136AF2E7E00E4FCFDABDE
:1024D60034AA33A932A831121EF9C8ECC8C9EDC90D
:1024E600CAEECACBEFCBE4FCFDFEEB2535F534EEA8
:1024F6003AF533ED39F532EC38F531AF34AE33AD6C
:1025060032FCAB39AA38A937A836D3121E99500324
:1025160002247F43300402247FE53020E003E48078
:102526002DE52C452D452B601EAB28E52A24FFF909
:10253600E52934FFFAEBC0E0EAC0E0E9C0E0AB2BE6
:10254600AA2CA92D121F58E53030E20774FFFFFEB2
:10255600FDFC22E530AF34AE33AD32AC3130E103B1
:04256600021E8B22A4
:101EE700BB010689828A83F0225002F722BBFE01DA
:021EF700F322D4
:101EF900E88FF0A4CC8BF0A42CFCE98EF0A42CFC88
:101F09008AF0EDA42CFCEA8EF0A4CDA8F08BF0A405
:101F19002DCC3825F0FDE98FF0A42CCD35F0FCEB64
:101F29008EF0A4FEA9F0EB8FF0A4CFC5F02ECD3929
:0F1F3900FEE43CFCEAA42DCE35F0FDE43CFC2296
:101F4800FAE6FB0808E6F925F0F618E6CA3AF6229A
:101F5800BB011A89828A83D0F0D0E0F8D0E0F9D0AA
:101F6800E0FAD0E0FBE8C0E0C0F0021FD65016E966
:101F7800F8D083D082D0E0F9D0E0FAD0E0FBC0827C
:101F8800C083021FCDBBFE16E9F8D083D082D0E013
:0F1F9800F9D0E0FAD0E0FBC082C083021FDF2245
:101FA700D083D082F8E4937012740193700DA3A3C9
:101FB70093F8740193F5828883E4737402936860DD
:061FC700EFA3A3A380DFDD
:091FCD00EBF608EAF608E9F62239
:091FD600EBF0A3EAF0A3E9F0220C
:091FDF00EBF208EAF208E9F22233
:00000001FF
